:020000040800F2
:1000000000180020CD1900080106000803060008AA
:1000100000000000000000000000000000000000E0
:1000200000000000000000000000000005060008BD
:100030000000000000000000070600080906000894
:100040004D1A00084D1A00084D1A00084D1A0008F4
:100050004D1A00084D1A00084D1A00084D1A0008E4
:100060004D1A00084D1A00084D1A00084D1A0008D4
:100070004D1A00084D1A00084D1A00084D1A0008C4
:100080004D1A000800000000000000004D1A000892
:10009000000000004D1A00084D1A00084D1A000813
:1000A000000000004D1A00084D1A00084D1A000803
:1000B0004D1A0008000000004D1A00084D1A0008F3
:1000C000002243088B4274D303098B425FD3030A97
:1000D0008B4244D3030B8B4228D3030C8B420DD3AA
:1000E000FF22090212BA030C8B4202D31212090238
:1000F00065D0030B8B4219D300E0090AC30B8B4276
:1001000001D3CB03C01A5241830B8B4201D38B0323
:10011000C01A5241430B8B4201D34B03C01A5241C8
:10012000030B8B4201D30B03C01A5241C30A8B420B
:1001300001D3CB02C01A5241830A8B4201D38B02F6
:10014000C01A5241430A8B4201D34B02C01A52419A
:10015000030A8B4201D30B02C01A5241CDD2C3090C
:100160008B4201D3CB01C01A524183098B4201D388
:100170008B01C01A524143098B4201D34B01C01A73
:10018000524103098B4201D30B01C01A5241C308EB
:100190008B4201D3CB00C01A524183088B4201D35A
:1001A0008B00C01A524143088B4201D34B00C01A46
:1001B0005241411A00D20146524110467047FFE7B2
:1001C00001B5002000F006F802BDC0460029F7D0B6
:1001D00076E770477047C04610B5064C2378002B71
:1001E00007D1054B002B02D0044800E000BF0123DB
:1001F000237010BD0C00002000000000A81A0008A9
:10020000044B10B5002B03D00349044800E000BFA5
:1002100010BDC0460000000010000020A81A000811
:1002200084B00F4B5A698021C9030A435A615A6945
:100230000A400192019A5A69802189020A435A614F
:100240005A690A400292029A5A698021C9020A43F5
:100250005A615B690B400393039B04B07047C0462F
:100260000010024072B6FEE700B585B00C220021F6
:1002700001A801F0ECFB1C481C4B03600023436009
:100280008360C360012202610421416103764376E9
:100290008376C376C221FF31C16103629E39FF3983
:1002A0004354826200F000FA002817D10023019322
:1002B00080235B01029380235B0503930A4801A915
:1002C00000F0B4FA00280BD101230193064801A9DC
:1002D00000F0ACFA002805D105B000BDFFF7C2FF61
:1002E000FFF7C0FFFFF7BEFF980000200024014089
:1002F00010B50B480B4B0360102343600023836051
:10030000C36003614361037643768376C3760377E4
:10031000437700F027FB002800D110BDFFF7A2FFB4
:10032000700000200064004000B58FB01022002152
:100330000AA801F08CFB0822002108A801F087FB25
:100340001C22002101A801F082FB2A488023DB0542
:10035000036000234360836001225242C260036154
:10036000836101F065F9002836D180235B010A938F
:1003700020480AA901F074FA00282FD11D4801F085
:1003800083F900282CD1002308930993194808A960
:1003900001F0EAFA002825D160230193002302939B
:1003A000039305931348002201A901F0D5F9002811
:1003B0001AD11048042201A901F0CEF9002815D164
:1003C0000C48082201A901F0C7F9002810D10948FA
:1003D00000F0DAF80FB000BDFFF744FFFFF742FF6F
:1003E000FFF740FFFFF73EFFFFF73CFFFFF73AFF45
:1003F000FFF738FF2800002010B592B0342200210A
:1004000005A801F024FB10241022002101A801F00E
:100410001EFB12230593113B08930A9309940B9436
:1004200005A800F059FC00280DD1072301930023F3
:10043000029303930493002101A800F02BFF0028EE
:1004400003D112B010BDFFF70DFFFFF70BFF10B582
:1004500000F008F9FFF7D0FFFFF7E2FEFFF704FF17
:10046000FFF746FFFFF760FFFEE7000082B00A4B90
:10047000996901221143996199690A400092009A91
:10048000DA69802149050A43DA61DB690B4001938F
:10049000019B02B07047C0460010024010B588B002
:1004A00004001422002103A801F0D1FA2268104BA5
:1004B0009A4201D008B010BD0E4B9A698021890084
:1004C0000A439A619A690A400192019A5A69802105
:1004D00089020A435A615B690B400293029B032322
:1004E00003930493902003A9C00500F037FBE1E7D4
:1004F000002401400010024010B588B0040014220E
:10050000002103A801F0A3FA2268134B9A4201D0FC
:1005100008B010BD114BDA69802189040A43DA6101
:10052000DA690A400192019A5A69802189020A43D4
:100530005A615B690B400293029BC0235B010393EA
:10054000022304930133069301330793902003A9F8
:10055000C00500F003FBDBE7006400400010024030
:1005600082B002688023DB059A4201D002B0704756
:10057000044AD16901231943D161D269134001931F
:10058000019BF3E70010024010B588B0040014226C
:10059000002103A801F05BFA22688023DB059A4260
:1005A00001D008B010BD144B5A69802189020A435A
:1005B0005A615A690A400192019A5A698021C90216
:1005C0000A435A615B690B400293029B2423039305
:1005D000022404940794902003A9C00500F0BEFAF9
:1005E000082303930494002305930693079403A917
:1005F000024800F0B3FAD4E70010024000040048BB
:10060000FEE7FEE77047704710B500F03BF810BDFD
:100610007047000010B504000F4B1978FA208000D5
:10062000FFF74EFD01000D4B1868FFF749FD00F084
:1006300091FA00280DD1032C01D901200AE00130E4
:1006400000222100404200F081FA054B1C6000208E
:1006500000E0012010BDC046040000200000002082
:100660000800002010B5064A136810210B431360E0
:100670000320FFF7CFFFFFF7F9FE002010BDC046B3
:1006800000200240034A1168034B1B785B1813607B
:100690007047C046D800002004000020014B1868B5
:1006A0007047C046D800002070B5041E00D1B4E0E9
:1006B000836B002B00D180E0A36BDB0600D5A6E0A6
:1006C00023689A68042108001040114200D09EE07F
:1006D000A26B53490A400631FF310A43A26399686D
:1006E00003220A40012A6ED0DA6818218A43A168E1
:1006F0000A43DA60226813699B009B0861680B4318
:1007000013612268D36847490B40D360237E9B0363
:10071000627ED2031343A17E4A031343A26A012AD5
:1007200058D0802252011343E26813432269022AFF
:1007300052D003432422A25C52001343E27E012ADA
:100740004CD0E269C221FF318A4202D0216A0A43B9
:1007500013432168CA681A43CA60E26A80214905C6
:100760008A420DD0012A0BD0022A09D0032A07D0D1
:10077000042A05D0052A03D0062A01D0072A0AD167
:100780002068416907229143416120684169E56A17
:100790002A400A4342612268D26823490A409A42A9
:1007A0002BD0A36B12229343023A1343A363E36B50
:1007B0000F3A1343E36301202EE0C36334228354D2
:1007C000FFF76CFE78E71A68D2079AD4DA68120449
:1007D00097D489E70200A6E70420AAE7002903D1FD
:1007E000802252021343ACE7A26B20210A43A2638A
:1007F000E26B1F390A43E263A3E70023E363A36BC1
:1008000003229343023A1343A363002004E0A36B43
:1008100010221343A363012070BD0120FCE7C046F2
:10082000FDFEFFFF1902FEFFE7FF3F8330B583B0F7
:100830000400002301933433C35C012B00D181E019
:1008400034230122C254026893685B076CD4486861
:100850003D4B98424DD0936A0D680120A840034358
:100860009362E36A072B27D8002B10D1886822688F
:10087000556907232B40984209D0506907239843B4
:100880005061206842698D682B40134343610B68B7
:100890001A00103A022A51D82C4A1268102B13D091
:1008A000112B0ED080235B041343284A13600B687E
:1008B000102B0CD000203CE0802252059342E6D061
:1008C000D4E78023DB03EFE780231B04ECE7204B16
:1008D00018682049FFF7F4FB83001B185B000193A5
:1008E00002E0019B013B0193019B002BF9D1002009
:1008F0001FE0936A0D680120A840834393620B6850
:100900001A00103A022A1BD8104A1268102B09D07C
:10091000112B05D0104B13400C4A1360002008E047
:100920000E4BF8E70E4BF6E7836B202213438363ED
:10093000012034230022E25403B030BD0020F8E748
:100940000020F6E70220F7E7011000000827014029
:100950000000002040420F00FFFFFFFEFFFFBFFF2F
:10096000FFFF7FFF70B5041E00D1A0E02023C35C11
:10097000002B1AD02268136801210B431360FFF784
:100980008DFE050022685368DB0711D4FFF786FE51
:10099000401B0A28F6D9626A80239B0213436362D4
:1009A00020230522E254012070BDFFF7A5FDE1E7F9
:1009B000136802218B431360FFF770FE0500226865
:1009C00053689B070ED5FFF769FE401B0A28F6D92E
:1009D000626A80239B021343636220230522E25450
:1009E0000120E1E7237E012B3ED0136880218B4359
:1009F0001360637E012B3CD02268136840218B4337
:100A00001360A37E012B3AD02268136820218B4308
:100A10001360E37E012B38D02268136810210B434A
:100A20001360237F012B36D02268136808218B4383
:100A30001360637F012B34D02268136804218B4339
:100A40001360A368E2681343226913436269134386
:100A50006268013A21681343CB610023636220334B
:100A60000122E25400209FE7136880210B431360AA
:100A7000BFE72268136840210B431360C1E7226877
:100A8000136820210B431360C3E722681368102109
:100A90008B431360C5E72268136808210B4313607A
:100AA000C7E72268136804210B431360C9E70120DC
:100AB0007AE7000070B5002811DB8308134DC033BE
:100AC0009B005C5903221040C000FC321600864097
:100AD000B44389010A40824022435A5170BD0F231A
:100AE0000340083B9B0806339B00094A9446634435
:100AF0005C6803221040C000FC3215008540AC4306
:100B000089010A40824022435A60E7E700E100E0A1
:100B100000ED00E0013880235B0498420FD2094ABF
:100B200050600948036A1B021B0AC02109060B43D7
:100B30000362002393600733136000207047012095
:100B4000FCE7C04610E000E000ED00E010B5FFF764
:100B5000B1FF10BD10B5FFF7DDFF10BDF0B583B0DC
:100B6000002356E086685F000324BC40A643CC689F
:100B7000BC4034438460446894434E683609012283
:100B800032409A402243426053E0DE080836B60005
:100B9000375805321A4092000F249440A7430C693D
:100BA000944022003A43325056E0022600E00026EC
:100BB000A64034003C4302329200424E9451424AD5
:100BC0009768EA433E00AE434C68E40201D53E001C
:100BD0002E433D4CA660E7683E0016404C68A402D8
:100BE00001D53E002E43384CE66067683E00164053
:100BF0004C68A40301D53E002E43334C6660266842
:100C000032404C68E40301D52A0032432E4C226066
:100C100001330C682200DA4051D001229A402500AD
:100C200015401442F4D04E6803243440013C012C9A
:100C300098D94C6803222240032A08D0C4685E0079
:100C40000322B24094438A68B2402243C2604C6897
:100C500003222240022A98D004685E000322170073
:100C6000B740BC434F683A40B240224302604C68F0
:100C7000C02292021442CBD0144CA6690122164322
:100C8000A661A46922400192019A9A08941CA400CA
:100C90000C4EA75903241C40A4000F26A640B743BE
:100CA0009026F605B04282D0094EB04205D0094EDA
:100CB000B04200D179E705267AE7012678E703B04C
:100CC000F0BDC04600000140000401400010024099
:100CD000000400480008004870B582B0041E00D12E
:100CE0007FE20368DB072BD5B34B5A680C23134014
:100CF000042B1DD0B04B5A680C231340082B0ED088
:100D00006368012B41D0002B56D1AB4B1A68AB491D
:100D10000A401A601A68AA490A401A603BE0A64BCA
:100D20005B68C02252021340802252029342E7D1F4
:100D3000A14B1B689B0303D56368002B00D153E2D2
:100D400023689B0777D59C4B5B680C221A4262D0C4
:100D5000994B5A680C231340082B53D0E368002B9F
:100D600000D18AE0944A136801210B431360FFF716
:100D700095FC0500904B1B689B0775D4FFF78EFC14
:100D8000401B0228F6D903202CE28B4A11688023ED
:100D90005B020B4313606368002B25D0FFF77EFCDA
:100DA0000500854B1B689B03CAD4FFF777FC401BEB
:100DB0006428F6D9032015E2052B09D07E4B1A686A
:100DC0007E490A401A601A687D490A401A60E2E7C3
:100DD000794B19688022D2020A431A60196880226E
:100DE00052020A431A60D6E7FFF758FC0500724B1F
:100DF0001B689B03A4D5FFF751FC401B6428F6D960
:100E00000320EFE16C4B5B68C0225202134080224A
:100E100012029342A2D1684B1B689B0703D5E3687B
:100E2000012B00D0E2E164490B68F8229343226968
:100E3000D20013430B6023681B0744D5E369002BE2
:100E40002ED05D4A536A01210B435362FFF726FC03
:100E50000500594B5B6A9B0735D4FFF71FFC401B0D
:100E60000228F6D90320BDE153490B68F8229343C9
:100E70002269D20013430B60DDE74F4A136801215A
:100E80008B431360FFF70AFC05004B4B1B689B0765
:100E9000D1D5FFF703FC401B0228F6D90320A1E1BE
:100EA000454A536A01218B435362FFF7F7FB050064
:100EB000414B5B6A9B0706D5FFF7F0FB401B0228FE
:100EC000F6D903208EE123685B0700D480E03A4B1B
:100ED000DB69DB001DD4384BDA69802149050A4300
:100EE000DA61DB690B400193019B0125354B1B68DF
:100EF000DB0510D5A368012B21D0002B36D12E4B5A
:100F00001A6A01218A431A621A6A03318A431A62F1
:100F10001AE00025EAE72B4A116880235B000B43A7
:100F20001360FFF7BBFB0600264B1B68DB05E1D413
:100F3000FFF7B4FB801B6428F6D9032052E11E4A58
:100F4000136A01210B431362A368002B24D0FFF71F
:100F5000A5FB0600184B1B6A9B0737D4FFF79EFBC7
:100F6000801B194B9842F5D903203BE1052B09D092
:100F7000114B1A6A01218A431A621A6A03318A43A1
:100F80001A62E1E70C4B1A6A04210A431A621A6AD0
:100F900003390A431A62D7E7FFF780FB0600064BC6
:100FA0001B6A9B0712D5FFF779FB801B064B984203
:100FB000F5D9032016E1C04600100240FFFFFEFFF6
:100FC000FFFFFBFF0070004088130000012D39D0A7
:100FD0002368DB0610D56369012B39D0053357D15F
:100FE000894A536B04218B435363536BF4318B4316
:100FF000A169C9000B43536323689B066ED5824BDE
:101000005A680C2313400C2B60D07F4B5A680C237A
:101010001340082B53D0236A002B7ED07A4A516BA1
:1010200080235B020B435363FFF738FB0500764BCD
:101030005B6B9B0352D4FFF731FB401B0228F6D9B0
:101040000320CFE0704AD36970490B40D361BFE7FA
:101050006D4B5A6B04210A435A635A6B03390A4396
:101060005A63FFF71BFB0500674B5B6B9B0706D4BE
:10107000FFF714FB401B0228F6D90320B2E06249B7
:101080004B6BF8229343A269D20013434B63B3E73F
:101090005D4B5A6B04210A435A635A6B03398A43E6
:1010A0005A63FFF7FBFA0500574B5B6B9B07A3D511
:1010B000FFF7F4FA401B0228F6D9032092E0524BC6
:1010C0005B68C022520213409342A4D14E4B5B6B2B
:1010D0009B0303D5236A012B00D089E0636A002BB0
:1010E00000D187E0484A51680C220A40082A60D0A3
:1010F000022B25D0444A136845490B401360FFF783
:10110000CDFA0400404B1B689B0150D5FFF7C6FA8F
:10111000001B0228F6D9032064E03B4A536B3D498B
:101120000B405363FFF7BAFA0500374B5B6B9B0329
:10113000D4D5FFF7B3FA401B0228F6D9032051E0BB
:10114000314A136832490B401360FFF7A7FA0500D4
:101150002D4B1B689B0106D5FFF7A0FA401B022808
:10116000F6D903203EE0284BDA6A0F218A43216B2F
:101170000A43DA625A6828490A40E16AA06A0143D0
:101180000A435A601968802252040A431A60FFF722
:1011900085FA04001C4B1B689B0106D4FFF77EFAFE
:1011A000001B0228F6D903201CE000201AE00020D2
:1011B00018E0012B20D0144B5A68D86AC0235B0278
:1011C0001340A16A8B4219D10F230340216B8B423C
:1011D00016D1F0239B031A40E36A9A4212D10020F1
:1011E00000E0012002B070BD0120FBE70120F9E71B
:1011F0000120F7E70020F5E70120F3E70120F1E700
:101200000120EFE70120EDE700100240FFFFFFEFB4
:10121000FFFFFFFEFFFFFEFFFF7FC2FF10B5184B71
:101220005A680C231340082B03D00C2B25D11548EA
:1012300010BD910C0F2319401348445C1049C96A32
:101240000B401249C95CC0235B021A4080235B0239
:101250009A4208D0C0235B029A4209D00C48FEF79C
:101260002FFF6043E4E70A48FEF72AFF6043DFE709
:101270000448FEF725FF6043DAE70548D8E7C04693
:1012800000100240006CDC02E01A0008D01A0008CE
:1012900000127A0070B504000D00002800D186E02D
:1012A000474B1A68012313408B420AD244490B680A
:1012B000012293432B430B600B681A40AA4200D0D3
:1012C00077E023689A070ED55B0705D53D4A51683C
:1012D000E023DB000B4353603A4A5368F0218B4311
:1012E000A1680B4353602368DB0735D56368012B86
:1012F00009D0022B24D0032B28D0324A126892073F
:1013000005D4012052E02F4A1268920353D52D498B
:101310004A680320824313434B60FFF7BFF906007E
:10132000284B5B680C221A4063689B009A4213D0DA
:10133000FFF7B4F9801B244B9842F1D9032035E024
:10134000204A12689201E2D401202FE01D4A526B1C
:101350009203DCD4012029E0194B1A6801231340C1
:10136000AB4209D916490B68012293432B430B600A
:101370000B681A40AA4220D123685B0706D5114AA0
:10138000536812490B40E1680B435360FFF746FF77
:101390000C4B5A6812090F2313400D4AD35CD840F6
:1013A0000C4B18600320FFF735F9002070BD0120B9
:1013B000FCE70120FAE70120F8E70120F6E7C04644
:1013C000002002400010024088130000FFF8FFFFD9
:1013D000C01A00080000002030B5036A01229343C0
:1013E0000362056A426883697324A3430C681C4343
:1013F00002239D438B682B43124DA84205D0124D0A
:10140000A84202D0114DA84206D10825AB431D00C9
:10141000CB682B430425AB430A4DA84205D00A4DA7
:10142000A84202D0094DA84205D1094D2A404D6974
:1014300015438A692A43426084614A6842630362B1
:1014400030BDC046002C014000440140004801402E
:10145000FFFCFFFF30B5036A164A13400362046ABB
:101460004268C3697325AB430D681D43124B1C4092
:101470008B681B022343114CA04206D0104CA042A3
:101480000AD0104CA0420FD106E00F4C1C40CB6894
:101490001B0223430D4C23400D4C22404C69240178
:1014A00014438A69120122434260C5614A68C263DB
:1014B000036230BDFFFEFFFFFFFDFFFF002C014078
:1014C0000044014000480140FFF7FFFFFFFBFFFF22
:1014D000FFCFFFFF30B5036A114A13400362046A6D
:1014E0004568C3690F4A13400A6812021A430E4B3B
:1014F0001C408B681B0323430C4CA04205D00C4CB2
:10150000A04202D00B4CA04204D10B4C2C404D69A0
:10151000AD0125434560C2614A680264036230BD83
:10152000FFEFFFFFFF8CFFFFFFDFFFFF002C0140FD
:101530000044014000480140FFBFFFFF30B5036A8F
:10154000046A0125AC4304628469EF35AC4312019F
:1015500022430A24A3430B438261036230BD00008F
:1015600030B5036A1024A34303628469036A054DFE
:101570002C4012032243A024A34309011943826192
:10158000016230BDFF0FFFFF8368702293430B435E
:10159000693A1343836070477047000003681E4A2E
:1015A000904206D08022D205904202D01B4A90423F
:1015B00003D1702293434A681343174A90420FD0D5
:1015C0008022D20590420BD0144A904208D0144A8F
:1015D000904205D0134A904202D0134A904203D160
:1015E000124A1A40CB681343802293434A6913433B
:1015F00003608B68C3620B688362074B984205D017
:10160000084B984202D0084B984201D10B69036302
:10161000012343617047C046002C01400004004094
:10162000002000400044014000480140FFFCFFFF53
:1016300070B5041E26D03D23C35C002B1CD03D2575
:1016400002236355210001C9FFF7A8FF01234622A9
:10165000A354083AA3540132A3540132A3540132D3
:10166000A3540132A3540132A3540132A3540132D2
:10167000A3546355002070BD3C330022C254FEF7D2
:101680006FFFDCE70120F6E770B5041E26D03D238E
:10169000C35C002B1CD03D2502236355210001C9EA
:1016A000FFF77CFF01234622A354083AA3540132DA
:1016B000A3540132A3540132A3540132A354013282
:1016C000A3540132A3540132A3546355002070BDCA
:1016D0003C330022C254FFF75FFFDCE70120F6E74E
:1016E00070B5036A102293430362026A45688369F6
:1016F000144C23400C6824021C4320239A438B681B
:101700001B011343104A904206D0104A90420BD05E
:101710000F4A904210D107E0802293431E00CB680D
:101720001B013343403A93430A4A15404A699200E9
:101730002A438D69AD001543456084614A68826320
:10174000036270BDFF8CFFFF002C0140004401408C
:1017500000480140FFF3FFFF70B504000D003C237B
:10176000C35C012B00D16AE03C230121C154082A4B
:1017700050D01CD8002A35D0042A16D10068290080
:10178000FFF7AEFF2268916980231B010B43936131
:10179000226893692B490B40936121688B692A6900
:1017A000120213438B61002030E001202EE00C2A4E
:1017B00016D100682900FFF78DFE2268D1698023C9
:1017C0001B010B43D3612268D3691E490B40D361CF
:1017D0002168CB692A6912021343CB61002015E00E
:1017E000012013E000682900FFF7F6FD22689369E5
:1017F00008210B4393612268936904398B439361F9
:101800002268936929690B43936100203C230022DD
:10181000E25470BD00682900FFF71CFE2268D369FE
:1018200008210B43D3612268D36904398B43D36108
:101830002268D36929690B43D3610020E6E70220BF
:10184000E7E7C046FFFBFFFF30B58468034D2C403F
:101850001B0213430B432343836030BDFF00FFFF94
:1018600010B504000B003C22825C012A00D177E015
:101870003C220121815401320131815401688A687E
:10188000384802408A60196860294FD023D840291F
:1018900057D011D8202904D00AD8002901D0102906
:1018A00004D12068FFF770FE00202AE0012028E024
:1018B0003029F6D0012024E050290AD15968DA688D
:1018C0002068FFF73BFE20685021FFF75DFE0020F7
:1018D00017E0012015E08022520191423CD0802285
:1018E0009201914214D0702938D199685A68DB6806
:1018F0002068FFF7A9FF2268936877210B43936064
:1019000000203D230122E254013B0022E25410BD9D
:1019100099685A68DB682068FFF796FF226891682B
:101920008023DB010B4393600020EAE75968DA6803
:101930002068FFF715FE20686021FFF725FE0020D4
:10194000DFE75968DA682068FFF7F8FD2068402172
:10195000FFF71AFE0020D4E70020D2E70120D0E7ED
:101960000220D4E78800FFFF30B53C23C35C012B85
:1019700025D03C230122C25401330132C2540368F2
:101980005C689D686E3294430A6822435A6003681B
:101990000C4A934206D08022D205934202D00A4AD2
:1019A000934204D1802295434A682A439A603D239A
:1019B0000122C254013B0022C254002030BD02204B
:1019C000FCE7C046002C0140000400401348854657
:1019D000FEF71EFE12480168090E124A914205D117
:1019E0001148124901601248124901601248134916
:1019F000134A002302E0D458C4500433C4188C4264
:101A0000F9D3104A104C002301E013600432A242C3
:101A1000FBD300F025F8FEF71AFDFEE700180020C2
:101A2000040000001F000000181002400100000028
:101A30000000014000000000000000200C00002019
:101A4000F81A00080C000020DC000020FEE703006C
:101A50008218934200D1704719700133F9E70000F2
:101A600070B500260C4C0D4D641BA410A64209D184
:101A7000002600F019F80A4C0A4D641BA410A64277
:101A800005D170BDB300EB5898470136EEE7B300BF
:101A9000EB5898470136F2E7F01A0008F01A0008F0
:101AA000F41A0008F01A0008F8B5C046F8BC08BCE3
:101AB0009E467047F8B5C046F8BC08BC9E467047C5
:101AC00000000000000000000102030406070809EE
:101AD0000102030405060708090A0B0C0D0E0F107E
:101AE00002030405060708090A0B0C0D0E0F10105F
:041AF00001020008E7
:041AF400D90100080C
:0C1AF80000127A00010000000400000051
:04000005080019CD09
:00000001FF
